:1000000042C05CC0DDC15AC059C058C057C056C0BC
:1000100055C054C053C052C051C050C04FC0B9CADF
:1000200065C8B6C8D4C8FDC82DC944C961C9A1C92D
:10003000A2C95AC8BFC9EDC9F0C954C851C886CAB7
:1000400004030904160355005300420074006900BC
:100050006E007900530050004900120110010000A9
:10006000000881179F0C0401000200010902190019
:1000700001010080640904000001FF000000070581
:1000800081030800640011241FBECFE5D2E0DEBF6B
:10009000CDBF10E0A0E6B0E0E0E2F6E102C00590DE
:1000A0000D92A636B107D9F710E0A6E6B0E001C080
:1000B0001D92AD3CB107E1F7C1D7B0CAA1CF1F93E4
:1000C000162F2091910024FF07C02091920038E85C
:1000D00023272093920003C02AE520939100212F2B
:1000E000DC01E3E9F0E08D91819321501216DCF3FD
:1000F00083E990E0612F4DD11C5F109391001F9117
:1001000008951F93CF93DF936091A200635067FD22
:10011000A7C080919F00CCE0D0E0C81BD109CA5590
:10012000DF4F80919E008D3209F088C0683009F061
:1001300095C083EC809386008AE5809360001092DE
:1001400066008881807631F0CE01DAD38F3F09F4E2
:1001500064C06AC09A8110928F008981882331F42B
:10016000109290002FE830E082E052C0853019F400
:100170009093A3004AC0863091F58B81813041F481
:100180008AE590E09093A1008093A00082E123C0D3
:10019000823041F48CE690E09093A1008093A0001F
:1001A00089E119C08330B1F4992341F480E490E0EF
:1001B0009093A1008093A00084E00DC0913051F095
:1001C000923041F484E490E09093A1008093A000E9
:1001D00086E101C080E090E49093660025C08830FD
:1001E00069F0893019F49093A5000FC08A3049F066
:1001F0008B3059F48BE48093920007C025EA30E0FD
:1002000002C02FE830E081E003C02FE830E080E05A
:100210003093A1002093A00007C0988197FD8E81A4
:1002200090E89093660007C09F81992321F49E81F6
:10023000981708F4892F8093610010C080916600A0
:1002400087FF0CC0CE010FD38F3F21F48EE1809346
:10025000600004C0882311F0109261001092A20087
:100260008091600084FF5BC0809161008F3F09F442
:1002700056C0182F893008F018E0811B8093610068
:100280008091860098E88927809386001123B1F138
:100290008091660087FF08C087E890E0612FC2D296
:1002A000182F8930B0F52AC02091A0003091A1000C
:1002B000412F415086FF0EC050E0EA01C857DF4F82
:1002C000F901A7E8B0E084918D933196AC17BD0792
:1002D000D1F70CC0D90150E0CA0188579F4FE7E819
:1002E000F0E06D916193E817F907D9F74F5F5F4F21
:1002F000420F531F5093A1004093A00087E890E065
:10030000612F47D01C5F1C3041F08FEF809361005C
:1003100004C08FEF809361001EE11093600084E1C0
:1003200096B3987131F48150D9F71092A3001092CE
:100330009D0011E0811110E080916700811729F084
:10034000112309F4F6D410936700DF91CF911F9128
:100350000895AC9A8BB780628BBF8BE48093920038
:100360008AE5809391000895A82FB92F80E090E04E
:1003700041E050EA609530E009C02D9182279795C1
:10038000879510F084279527305EC8F36F5FA8F338
:100390000895EADF8D939D930895A6E08827992715
:1003A000AA9569F00197E1F3B399FCCFB39BFECF17
:1003B00081E09927A6B3019611F0A871D9F70895A5
:1003C000CF93CFB7CF93C395B39BE9F7B39B0BC044
:1003D000B39B09C0B39B07C0B39B05C0B39B03C0CD
:1003E000B39B01C0D5C00F92DF93C0919F00DD2762
:1003F000CA55DF4F012EB39B03C0DF910F90E6CFAC
:100400002F930F931F934F932FEF4F6F06B303FB61
:1004100020F95F933F9350E03BE065C016B301269F
:10042000502953FDC89556B3012703FB25F92F73B7
:1004300006B3B1F05027102713FB26F906B222307D
:10044000F0F000C016B3012703FB27F9012650295D
:1004500006B22430E8F54F77206816B30000F6CFD7
:1004600050274F7D206206B2102F000000C006B357
:1004700000265029102713FB26F906B2E2CF4F7B46
:1004800006B3206400C0DACF01265029187106B2E5
:1004900069F14E7F2160012F16B328C00026502934
:1004A0004D7F06B22260102F29C0012650294B7FB4
:1004B00006B22460012F2DC016B301265029477FB4
:1004C0002860000006B22EC04F7E06B3206130C007
:1004D000422706B3499300265029102706B24FEF52
:1004E00013FB20F9297F16B379F2187159F101260F
:1004F000502906B2012703FB21F9237F06B371F2CD
:10050000002650293150D0F006B2102713FB22F9F3
:10051000277E16B351F201265029012703FB06B2AC
:1005200023F92F7C49F2000006B3102713FB24F9AE
:100530000026502906B22F7939F270CF10E21ABF87
:10054000002719C03B503195C31BD04010E21ABFA1
:100550000881033C09F10B34F9F020919D001981C9
:10056000110F1213EDCF4A81441F093651F10D329C
:1005700011F0013E29F70093A4003F915F914F9144
:100580001F910F912F91DF910F90CAB7C5FD1BCF1F
:10059000CF91CFBFCF9118952091A400222369F36A
:1005A0001091A200112379F534307AF13093A20032
:1005B00020939E0010919F003BE0311B30939F00E1
:1005C00024C00091A2000130F4F40AE54F7049F410
:1005D0003091600034FD1AC000936000C6E8D0E09E
:1005E00019C03091910034FD11C000939100C2E90F
:1005F000D0E010C0052710E000C021C0052710E0A2
:10060000C89508BB14C03AE501C032ED032EC0E026
:10061000D0E032E017B31861C39A08B317BB58E1B2
:1006200020E84FEF20FF052708BB279517951C3FB3
:1006300028F700004552B0F720FF0527279508BB93
:1006400017951C3FB8F629913A9561F7077E1091EE
:10065000A300110F08BBC250D04011F010939D00B1
:1006600010E21ABF086017B3177E402F477E54E090
:100670005A95F1F708BB17BB48BB7FCFFC015091DF
:100680006500862F972FDC0194E0619128E030E02F
:1006900040E880E0742F762309F0C09A052E00C050
:1006A0000000000000000A94D1F7C29A052E00C095
:1006B0000000000000000A94D1F7880FB1998F5F05
:1006C000C098C29846952150304021F78D939150A3
:1006D000E1F6089580917800909179009C012F5F58
:1006E0003F4F309379002093780020917A0027FFC4
:1006F00002C0880F991F20937E0080FF03C02860EE
:1007000020937E00292F269520937F00969587952C
:10071000809380008EE790E062E870E0AFDF08959C
:10072000B99A24E030E0E1E09E2F982321F098B3BD
:100730009C7F926002C098B39C7F98BBEE0F109292
:10074000750007C045E04A95F1F700C09F5F9093A0
:10075000750090917500692F70E040916300509191
:1007600064006417750770F3C09A1092750007C093
:1007700045E04A95F1F700C09F5F90937500909116
:100780007500692F70E04091630050916400641718
:10079000750770F32150304039F688B38C7F88BBE1
:1007A0000895B99A28E030E0E1E09E2F982321F0E7
:1007B00098B39C7F926002C098B39C7F98BBEE0F69
:1007C0001092750007C045E04A95F1F700C09F5FA1
:1007D0009093750090917500692F70E040916300CF
:1007E000509164006417750770F3C09A10927500F9
:1007F00007C045E04A95F1F700C09F5F90937500F0
:1008000090917500692F70E04091630050916400F1
:100810006417750770F32150304039F688B38C7F28
:1008200088BB0895EF92FF921F93DF93CF930F92AF
:10083000CDB7DEB7182F862F612F792F7B0108C027
:10084000898348DF90918500F70191937F01898129
:100850009E2D911B9817A0F30F90CF91DF911F91C0
:10086000FF90EF900895DF92EF92FF920F931F9306
:10087000CF93DF93F82EE62E0F2D192F50E6D52EAD
:1008800032C0F80181918F018093810023DF809134
:100890007E008D2580937E00C0E0D0E01DC08EE7F5
:1008A00090E062E870E0EADE80918500909181003E
:1008B000891741F490917600891721F09091770083
:1008C000891789F42091650030E045E0220F331F3D
:1008D0004A95E1F7C20FD31F20917B0030917C0035
:1008E000C217D307E0F2802F8F198E1550F281E0E6
:1008F000DF91CF911F910F91FF90EF90DF900895BE
:10090000CF93DF93EC014981442341F481E2898351
:10091000D093A100C093A00088E008C2413011F438
:1009200086B307C15A81423011F458BBFEC102960A
:10093000652F677021E030E0062E02C0220F331FC2
:100940000A94E2F7433029F498B3822F80958923E3
:1009500093C0443019F488B3822B8EC0453049F4DB
:1009600050936500B99887B3856287BB88B3887D4B
:1009700083C0463049F4B898C098B998C098BA98DE
:10098000C09880E287BB78C0473041F4BE0176DE74
:10099000D093A100C093A00084E0C8C1483031F4D6
:1009A000509376008B8180937700BFC18C819D81AD
:1009B0009093790080937800493011F480E211C05F
:1009C0004B3011F480EA0DC08A819B8190937C00AA
:1009D00080937B004A3011F480E403C04C3029F44A
:1009E00080EC80937A008FEFA1C14D3029F487B35A
:1009F0002095282327BB99C14E3021F487B3822B41
:100A000087BB93C14F3009F5552329F480917D00B0
:100A100087B9A59A0CC0513031F480917D00816076
:100A200087B9A29A04C0523011F48FE887B9369A78
:100A30003699FECF84B1888385B18983D093A10094
:100A4000C093A00014BA82E071C1403159F4B89A41
:100A5000B99A8AB5806A8ABD8AB583608ABD83B730
:100A6000856038C0413121F459BD8C8188BD5DC19C
:100A7000423121F488B3822B88BB57C1433129F41A
:100A800088B32095282328BB50C1443151F486B344
:100A900090E08223932302C0959587956A95E2F7AB
:100AA00048C0463169F5552319F483B78B7F24C0BC
:100AB000513031F483B78B7F83BF83B7826013C01B
:100AC000523051F483B78B7F83BF83B7826083BF7B
:100AD00083B7816083BF29C1533049F483B78460F1
:100AE00083BF83B78D7F83BF83B78E7FF3CF5430AF
:100AF00009F01BC183B7846083BF83B78D7FE7CFC5
:100B00004F3149F49B8180E0850F911D90936400E3
:100B1000809363000AC1403219F41ABC13BE05C1A8
:100B2000413221F45093C50081E0B5C0423241F416
:100B300081E18883D093A100C093A00081E0F6C03A
:100B40004332D9F4379A86B19A81892B86B98B8141
:100B5000813049F0813020F0823009F0E6C007C0D2
:100B600010927D00E2C080917D00806803C080917A
:100B70007D00806980937D00D8C0483249F48CEBB9
:100B800090E09093A1008093A0008091C400CEC01B
:100B9000493211F482E07FC04A3211F483E00BC085
:100BA0004B3211F484E077C04C3211F488E073C00A
:100BB0004D3239F489E0809368008A818093C500C2
:100BC000B4C04E3259F48BE0809368008A818093E0
:100BD000C5008B818093C6008C8134C04F3259F49C
:100BE000513031F4B89AB99ABA9A509374009DC0B2
:100BF000109274009AC0403349F450936E008B8178
:100C000080936F008C81809370008FC0413329F4F2
:100C10005093690010926A0088C0423311F485E055
:100C20003AC0433321F45093C50086E034C04433C6
:100C300061F4509368008B818093C5008C81809310
:100C4000C6008D818093C70070C0453369F450930E
:100C5000C5008B818093C6008C818093C7008D81F5
:100C60008093C80080E117C0842F90E0807F90704F
:100C7000803D910599F447704093C5008A81809327
:100C8000C6008B818093C7008C818093C8008D81C2
:100C90008093C9008EE08093680047C0803E910534
:100CA00001F58AE080936800842F87708093C500E7
:100CB00048704093C6001092750080E00BC090E031
:100CC0000296FE01E80FF91F30818B539F4FFC0104
:100CD0003083822F9091C500282F2F5F891778F3DA
:100CE00022C0803F910509F587E080936800842F3A
:100CF00088708093C50047704093C60010927500BD
:100D000080E00BC090E00296FE01E80FF91F3081F1
:100D10008B539F4FFC013083822F9091C600282F68
:100D20002F5F891778F38093750080E0DF91CF9172
:100D30000895DF92EF92FF920F931F93CF93DF936B
:100D4000C8E0D0E0FF2460E8E62EDE2CDF0CD1BE48
:100D500024DB082F192F89E0043318070CF4FD2C2D
:100D6000E694219791F78F2D815081BFCF2DD0E050
:100D7000219610C012DB8453994097FF03C09095D1
:100D800081959F4F8017910714F4F1B68C0181B7BC
:100D90008F5F81BF81B790E0C817D9075CF7F1BEBC
:100DA00061B780E090E02CD4DF91CF911F910F913B
:100DB000FF90EF90DF900895882311F0B99801C05B
:100DC000B99ABA981092750007C025E02A95F1F7F4
:100DD00000C09F5F9093750090917500492F50E07F
:100DE0002091690030916A004217530770F3BA9A54
:100DF0001092750007C025E02A95F1F700C09F5FAB
:100E00009093750090917500492F50E020916900F2
:100E100030916A004217530770F38111B99A08950F
:100E2000B998BA981092750007C025E02A95F1F795
:100E300000C04F5F4093750040917500242F30E053
:100E40008091690090916A002817390770F386B382
:100E5000BA9A1092750007C025E02A95F1F700C0F4
:100E60009F5F9093750090917500492F50E02091FD
:100E7000690030916A004217530770F386958170BC
:100E8000089588B3897F88BBBA98B9981092750085
:100E900007C085E08A95F1F700C04F5F4093750069
:100EA00040917500242F30E08091690090916A0094
:100EB0002817390770F3089587B3897F87BB10928D
:100EC000750007C085E08A95F1F700C04F5F409339
:100ED000750040917500242F30E080916900909159
:100EE0006A002817390770F3B99A1092750007C085
:100EF00085E08A95F1F700C04F5F409375004091FF
:100F00007500242F30E08091690090916A002817C5
:100F1000390770F3BA9A1092750007C085E08A9578
:100F2000F1F700C04F5F4093750040917500242F8A
:100F300030E08091690090916A002817390770F3BA
:100F40000895B99ABA9A1092750007C085E08A95FB
:100F5000F1F700C04F5F4093750040917500242F5A
:100F600030E08091690090916A002817390770F38A
:100F7000BA981092750007C085E08A95F1F700C015
:100F80004F5F4093750040917500242F30E08091B1
:100F9000690090916A002817390770F3B998109288
:100FA000750007C085E08A95F1F700C04F5F409358
:100FB000750040917500242F30E080916900909178
:100FC0006A002817390770F308950F931F93082FAD
:100FD00018E0802F8078F0DE000F1150D1F720DF6D
:100FE0001F910F910895FF920F931F93F82E08E021
:100FF00010E0110F15DF182B0150D9F7FF2011F069
:1010000080E001C081E0D8DE1092750007C095E055
:101010009A95F1F700C08F5F8093750080917500FD
:10102000482F50E02091690030916A004217530721
:1010300070F3812F1F910F91FF900895DF92EF922F
:10104000FF920F931F93CF93DF9380E287BB88BB00
:1010500080E090E0CDD28F3F09F081BFBB9A84E160
:10106000E2EBF1EF3197F1F700C000008150C1F7DA
:10107000BB9885E090E090936A008093690010929D
:101080006400109263002EE088E190E00FB6F894BF
:10109000A89581BD0FBE21BD10926B0010926C000F
:1010A00010926D0010926E0010926F0010927000FE
:1010B00010927100109268004CD97894BBE1EB2E2D
:1010C000AAE1FA2E00E410E8A8951BD8E091680088
:1010D000F0E0E131F10508F05AC2E15FFF4F0994F9
:1010E00060E02AC2DD24D9C1DD2457C1B89AB9987D
:1010F000BA9AC29A1092BC008091C5008093720087
:10110000109373003FC0C09840E005C0F5E0FA9529
:10111000F1F700C04F5F242F30E080916300909181
:1011200064002817390790F3809173009091720042
:10113000892309F0C09AC2988091BC00880F8093DF
:10114000BC002091BC0086B390E0827090709595B1
:101150008795280F2093BC0040E005C025E02A9524
:10116000F1F700C04F5F242F30E080916300909131
:1011700064002817390790F3C29A8091730086950E
:101180008093730080917300882309F0BCCF1DC049
:10119000BA9AC2988BEB97E00197F1F700C0000074
:1011A0009FB7F894C29AE0E2F1E03197F1F700C0FE
:1011B000BA9881E0B29980E08093BC009FBF8BE930
:1011C00096E00197F1F7BA9AC29A81E0BCC180918A
:1011D000C50080937300BA9A88E02FB7F894C2983C
:1011E0009091730090FF0BC091E29A95F1F7C29A2B
:1011F000E7E0F1E03197F1F700C0000009C0E7EF48
:10120000F0E03197F1F70000C29AF7E3FA95F1F7B1
:10121000909173009695909373002FBF8150E9F6DB
:10122000B6C11092BC0028E08091BC0086958093E6
:10123000BC00BA9A3FB7F894C29881E28A95F1F758
:10124000C29A97E39A95F1F7BA9886B390E08470C2
:1012500090709595879595958795809373003FBF7E
:10126000E2EEF0E03197F1F700C0000080917300EA
:10127000882329F08091BC0080688093BC002150B5
:1012800099F6A3CFBA9A2FB7F894C298F1E2FA95DB
:10129000F1F7C29A87E38A95F1F7BA9886B390E09E
:1012A0008470907095958795959587958093BC00EF
:1012B0002FBF8BCFBA9A8FB7F894C2989091C50080
:1012C00090FF0BC091E29A95F1F7C29AE7E0F1E046
:1012D0003197F1F700C0000009C0E7EFF0E0319767
:1012E000F1F70000C29AF7E3FA95F1F78FBF4FC10B
:1012F000B99AB898BA9AC298E0927200FDB88091F3
:10130000C5008111C5981092730026C0F0E0E95322
:10131000FF4F80818FB90EB9809172008DB940E086
:1013200005C025E02A95F1F700C04F5F242F30E07B
:1013300080916300909164002817390790F3769BA1
:10134000EBCF80917300E82FF0E09FB1E454FF4FA2
:1013500090838F5F80937300E09173008091C6004B
:10136000E817A0F28091C5008111C59AE093C400EE
:101370000EC187DD0CC180E090E09EDD8091C5004C
:1013800024DE8093730013C0ED2DF0E0E953FF4F8E
:1013900080811BDE80937300D3948091C500D816A2
:1013A00098F38091C6008111CCDD80917300809309
:1013B000BC000BCF8091C500882311F4DD241EC032
:1013C000DD2404C081E00FDE8883D3942D2D30E02E
:1013D0008091C60090E00197E901C454DF4F2817BF
:1013E000390784F380E0FFDD88830CC0CD2DD0E089
:1013F00081E0F9DDC454DF4F8883D3948091C60027
:10140000D816A0F38091C700882309F49AC099DD0B
:1014100098C08091C60084D9BAC04091C600B99ADC
:101420002FC088B38C7F88BB41501092750007C0D5
:1014300085E08A95F1F700C05F5F50937500509189
:101440007500252F30E0809163009091640028178B
:10145000390770F3C09A1092750007C095E09A950D
:10146000F1F700C05F5F5093750050917500252F14
:1014700030E080916300909164002817390770F381
:10148000442379F688B38C7F88BB81C0ED2DF0E0D2
:10149000EA53FF4F808185D9D3948091C500D81637
:1014A000A8F375C0B998C19A88E090E071E01092F5
:1014B000750007C0F5E0FA95F1F700C0EF5FE09323
:1014C0007500E09175004E2F50E02091630030913F
:1014D00064004217530770F3C09A1092750007C05A
:1014E00025E02A95F1F700C0EF5FE0937500E091E9
:1014F00075004E2F50E02091630030916400421738
:10150000530770F330917300B19B04C0372B3093B5
:10151000730005C0272F2095232320937300C098C4
:10152000770F019721F6C198E62FF0E080917300C4
:10153000E454FF4F80836F5F8091C600681708F402
:10154000B1CF8091C6008093C40021C080E0E8D86C
:101550008091C60026D98091C70023D98091C80008
:1015600020D9109273000DC080E0DAD880E019D93C
:1015700080E017D980E015D9809173008F5F809348
:1015800073008091C50090917300981768F31092D2
:10159000680080917400882309F496CD80917100D1
:1015A000882369F490916E0090936B0090916F0086
:1015B00090936C009091700090936D0015C0909185
:1015C0006B00981710F4C09801C0C09A90916C00FD
:1015D000981710F4C19801C0C19A90916D009817A6
:1015E00010F4C29801C0C29A8F5F809371006CCDD5
:1015F000E199FECF9FBB8EBBE09A99278DB30895EA
:10160000262FE199FECF1CBA9FBB8EBB2DBB0FB618
:10161000F894E29AE19A0FBE01960895F894FFCFEC
:061620005AFF110A002828
:00000001FF
